:020000040000FA
:040000008A110F282A
:10000800FE00030EF9000A08FA00831203137F08A2
:10001800FB008A11EB298A111128F001F101F20184
:10002800F301F401F501F601F70183120313A001AE
:10003800A10183018A1120288316031381138312D7
:1000480003131F108316031708108810081188114E
:1000580008120910891009118911091289128316C9
:10006800031306148614061586150612861206133F
:1000780086130710871007118711071287120713B5
:1000880087138510051185110512851281128115B6
:100098000114811401158B168B17D629771C582843
:1000A8008312031306165B288312031306127708BC
:1000B800A20001300310A20CFF3E031D5E28221C83
:1000C80069288312031386166C2883120313861279
:1000D8007708A20002300310A20CFF3E031D6F2810
:1000E800221C7A288312031306177D288312031310
:1000F80006137708A20003300310A20CFF3E031D6D
:100108008028221C8B288312031386178E288312BB
:10011800031386137708A20004300310A20CFF3ED5
:10012800031D9128221C9C288312031307149F285F
:100138008312031307107708A20005300310A20CDE
:10014800FF3E031DA228221CAD2883120313871427
:10015800B028831203138710761CB6288312031362
:100168000715B9288312031307117608A200013076
:100178000310A20CFF3E031DBC28221CC7288312B3
:1001880003138715CA288312031387117608A20060
:1001980002300310A20CFF3E031DCD28221CD828D4
:1001A800831203130716DB2883120313071276083A
:1001B800A20003300310A20CFF3E031DDE28221C00
:1001C800E928831203138716EC2883120313871276
:1001D8007608A20004300310A20CFF3E031DEF288E
:1001E800221CFA28831203130717FD28831203130E
:1001F80007137608A20005300310A20CFF3E031D6A
:100208000029221C0B298312031387170E29831236
:1002180003138713861D63297508A2002208F400BA
:100228000D307502031C1B290C30F40222297508B5
:10023800031D22290C30A2002208F400741C28296E
:100248008312031385142B29831203138510740852
:10025800A20001300310A20CFF3E031D2E29221C10
:1002680039298312031305153C2983120313051139
:100278007408A20002300310A20CFF3E031D3F29A0
:10028800221C4A298312031385154D29831203134F
:1002980085117408A20003300310A20CFF3E031D51
:1002A8005029221C5B298312031305165E29831229
:1002B800031305120C3075020318AB29AF29751CFE
:1002C80069298312031385146C298312031385107B
:1002D8007508A20001300310A20CFF3E031D6F2910
:1002E800221C7A298312031305157D29831203130F
:1002F80005117508A20002300310A20CFF3E031D71
:100308008029221C8B298312031385158E298312B9
:10031800031385117508A20003300310A20CFF3ED9
:10032800031D9129221C9C298312031305169F295A
:100338008312031305127508A20004300310A20CDF
:10034800FF3E031DA229221CAD2983120313851623
:10035800B0298312031385128618C32972087304FF
:10036800031DC329E830F2000330F3000130A20076
:100378002208F507183075020318F501F701061968
:10038800D62970087104031DD629E830F00003301F
:10039800F1000130A2002208F6073C30760203186B
:1003A800F601F7018312061C52280612861206135C
:1003B8008613071087100711871107128712071372
:1003C800871385100511851105128512D6290B1D75
:1003D8003F2A0130A0070318A10A0030A10721080D
:1003E800803AFF008F307F02031DFC29FF30200276
:1003F800031C1C2A83120313A001A1010130F80079
:100408007808F7073C307702031C1C2AF7010130F3
:10041800F8007808F6073C307602031C1C2AF6011F
:100428000130F8007808F507183075020318F5014F
:100438007308803AFF0080307F02031D252A0130AF
:100448007202031C2D2AFF30F2070318F30AFF304B
:10045800F3077108803AFF0080307F02031D362AB7
:1004680001307002031C3E2AFF30F0070318F10A1E
:10047800FF30F1070B117B0883120313FF007A0882
:0C0488008A00790E8300FE0E7E0E090033
:04400E00F1E3FFFFDC
:00000001FF
